:020000001C0AD8
:08000800A304AB0AA304A80A3B
:10001000A304A60AA304A40AA304A20AA304A00A90
:10002000A3049E0AA3049C0AA304990AA304970AA2
:10003000A304810AA304790AFF0C28000905A3047C
:1000400008092905A3040A094905A3040C0969053F
:10005000A3040E098904A3041009A904A304120926
:10006000BF0C2C00A30404096B00A3040607450A77
:10007000A3042607450AA3044607450AA304660706
:10008000450A020C2C00A3041A09A30406064C0A14
:10009000040C2C00A3041A09A3042606530A080C16
:1000A0002C00A3041A09A30446065A0A100C2C00BB
:1000B000A3041A09A3046606610A200C2C00A304F9
:1000C0001A09C80C8B00A3040306750A8A05A30449
:1000D0001609010C2C00A3041A098A04A3041609AA
:1000E000010C2C000B02CC012B00A304350AA30445
:1000F000770A0C022D00640C2E00640C2F00A30460
:10010000180AFF0CA40430000E0232000D02310068
:10011000170CA304D00103068A0AA304F102880A7B
:10012000A304F202860AA304EF02840A0008A304CF
:10013000140A0A0226000008A304060AA304060AF9
:10014000A304060AA304060AA304060AA304060AD3
:0C0150000902060000080C020200000872
:021FFE000A00D7
:00000001FF
